:020000040800F2
:10000000F81F0020010100083F110008C30F00087D
:100010003D110008D3060008A520000800000000DC
:10002000000000000000000000000000E1110008D6
:100030001107000800000000DF1100081518000873
:100040001B0100081B0100081B0100081B01000820
:100050001B0100081B0100081B0100081B01000810
:100060001B0100081B0100081B0100081B01000800
:100070001B0100081B0100081B0100081B010008F0
:100080001B0100081B0100081B0100081B010008E0
:100090001B0100081B0100081B0100081B010008D0
:1000A0001B0100081B0100081B0100081B010008C0
:1000B0001B0100081B010008000000001B010008D4
:1000C0001B01000800000000000000001B010008E8
:1000D00000000000852000089520000800000000B6
:1000E0001B0100081B0100081B010008DFF80CD0F1
:1000F00000F06EFA00480047ED200008F81F0020CD
:100100000648804706480047FEE7FEE7FEE7FEE7B1
:10011000FEE7FEE7FEE7FEE7FEE7FEE779190008E7
:10012000ED0000082DE9F05F0546002092469B4651
:1001300088460646814640241BE0284641464746FD
:10014000224600F020F853465A46C01A914110D377
:1001500011461846224600F073F82D1A67EB010885
:100160004F4622460120002100F06AF817EB0009F3
:100170004E41201EA4F10104DFDC484631462A46E8
:100180004346BDE8F09F202A04DB203A21FA02F022
:100190000021704721FA02F3D040C2F120029140C1
:1001A00008431946704740EA01039B0703D009E062
:1001B00008C9121F08C0042AFAD203E011F8013B53
:1001C00000F8013B521EF9D27047D2B201E000F8AC
:1001D000012B491EFBD270470022F6E710B51346EB
:1001E0000A4604461946FFF7F0FF204610BD00F00E
:1001F000004230F000400AD0C10D01F56071C0F33B
:10020000160042EA0151C20840071143704700201E
:100210000146704730B50B460146002020220124DC
:1002200009E021FA02F59D4205D303FA02F5491BC4
:1002300004FA02F52844151EA2F10102F1DC30BDDA
:10024000202A04DB203A00FA02F100207047914096
:10025000C2F1200320FA03F31943904070472DE9BF
:10026000FE4F804681EA0300C00F0C46009021F04B
:10027000004123F00045B8EB0200A94105D24046F9
:10028000214690461C460B46024623F00040104390
:1002900047D0270DC7F30A00C3F30A510290401A52
:1002A000019040286BDAC3F3130040F4801B0098E0
:1002B000924620B10023D2EB030A63EB0B0B0198AB
:1002C0005946C0F140025046FFF7BAFF06460D46B8
:1002D00050465946019A00F08DF910EB0800614133
:1002E000002487EA115284EAE7731A4340D0009A47
:1002F00062B3019A012A4FEA075215DC001B61EB39
:1003000002014FF0004202EA0752CDE90042001C10
:1003100041F5801132462B4600F08DF903B0BDE85F
:10032000F08F40462146F9E7001B61EB0201001CFB
:1003300041F5801300185B412018A2F5001747EB28
:10034000030140EAD570B6196D4111E06D084FEA1E
:10035000360645EAC0754FEA0752001B61EB020101
:10036000001C41F5801149084FEA30000019514145
:1003700032462B4603B0BDE8F04F00F04DB900986F
:10038000012240000023D0EB020263EBE0730098EF
:1003900021464FEAE074B8EB000061EB0401E9E7A5
:1003A00083F000435BE781F0004158E72DE9FE4F01
:1003B00081EA030404F0004421F0004100944FF06E
:1003C000000B23F0004350EA01045ED052EA03041C
:1003D0005BD0C3F30A54C1F30A552C44A4F2F3349E
:1003E0000194A0FB0254C1F3130141F48011C3F343
:1003F000130343F4801301FB024400FB034E840A01
:10040000970A44EA815447EA8357A4FB0768029598
:100410008D0A05FB07854FEA932C04FB0C54270536
:10042000029D4FEA065847EA1637B5EB08056EEB12
:10043000070C870E920E47EA811742EA8312A7FB48
:100440000201B6EB0B0164EB00042B0D43EA0C3305
:100450005E1844EB1C50DA465146E7FB0201C5F337
:1004600013044FEA0B3343EA14534FEA0432019C5E
:1004700043EA0603A4F10C040294009CCDE900B405
:1004800000F0D9F803B0BDE8F08F00200146F9E78D
:100490002DE9F04D81EA030404F0004B21F0004502
:1004A00014464FF0000A23F0004150EA050220D024
:1004B00054EA01021DD0C5F30A570246C5F31303DF
:1004C000C1F31300C1F30A5640F4801543F48013BE
:1004D000A7EB0608101BD64608F2FD3873EB0500A3
:1004E00002D308F1010801E092185B41B8F1000F56
:1004F00003DA00200146BDE8F08D00204FF48011A2
:10050000064684460EE0171B73EB050705D3121B46
:1005100063EB050306434CEA010C49084FEA30003F
:1005200092185B4150EA0107EDD152EA030012D064
:1005300082EA040083EA0501084305D0101BAB41A1
:1005400006D20122002306E000224FF0004302E021
:100550006FF0010253101AEB06004CEB085110EB40
:100560000A0041EB0B01BDE8F04D00F055B8C1F3B6
:100570000A52C1F3130140F2FF3341F480119A4251
:1005800002DA00200146704740F233439A42A2F259
:10059000334202DC5242FFF7F6BDFFF751BE0000C6
:1005A00030B5041E71F1000404DB4FF000444042FA
:1005B00064EB0101141E73F1000405DB1C464FF0CF
:1005C0000043524263EB0403994208BF904230BD9E
:1005D000064C074D06E0E06840F0010394E8070090
:1005E00098471034AC42F6D3FFF784FD882C0008FE
:1005F000A82C0008202A06DBCB17203A41FA02F08B
:1006000043EAE07306E041FA02F3D040C2F120026F
:10061000914008431946704710B5141E73F1000449
:1006200008DA401C41F1000192185B411A4301D1E4
:1006300020F0010010BD2DE9F04D92469B4611B10E
:10064000B1FA81F202E0B0FA80F220329046FFF770
:10065000F7FD04460F4640EA0A0041EA0B01534603
:100660005A46084313D0114653EA010019D0C8F185
:1006700040025046FFF787FD05460E465046594654
:100680004246FFF7DDFD084305D0012004E0204687
:100690003946BDE8F08D0020054346EAE0762C435C
:1006A00037430A986305E40AA0EB08000022FD0A1C
:1006B00044EA47540A3002D500200146E9E7010523
:1006C00010196941DDE9084500196941BDE8F04D9F
:1006D000A2E7FEE782B08DF803009DF8030030B971
:1006E000FFE740F6A010C2F2000001900DE09DF877
:1006F0000300012806D1FFE740F6C410C2F2000053
:10070000019002E000200190FFE7019802B07047DD
:100710007047000070B1012808BF0220012181F359
:1007200010880549C8600020887080F31088887898
:100730000128FCD1704700BF10000020B0B50B4964
:10074000BD4B0B4C0A681B68B3FBF4F34C68584371
:1007500000234D68AC42FCD023445B1BAC4298BFE5
:1007600013442C46834228BFB0BDF2E714E000E0FA
:1007700040420F0081B080480222016841F001012F
:100780000160006800F001000090009803480168D3
:1007900062F31A61016001B0704700BF04000140BC
:1007A000012001F00FB9012001F024B97047014682
:1007B000012001F037B90A460146012001F030BAA4
:1007C0000A46014601A001F095FDFEE74572726FF1
:1007D00072206F636375727265643A2066696C6536
:1007E000202573206F6E206C696E652025640D0ACC
:1007F000000000002DE9FC4F5C4A03234FF0000A83
:100800004FF001084FF00F0C4FF00009904208BF65
:100810000223009300250B6833FA05F208BFBDE8F8
:10082000FC8F08FA05FE13EA0E0F00F09A804F685D
:10083000032F16D9112F26D0122F28D04F4A9742B6
:1008400013D04F4A974210D04E4A97420DD04E4A8D
:1008500097420AD04D4A974207D04D4A974204D05A
:1008600022E0DFE807F002181B1F8B6843B1012B61
:1008700014BFC0F814E0C0F810E04FF0080913E00E
:100880004FF0040910E0CB6803F104090CE0CB68D9
:1008900003F10C0908E0D1F80C9005E0CB6803F1F6
:1008A000080901E04FF0000953460646082D28BF0D
:1008B000203B28BF043637680CFA03F409FA03F327
:1008C00027EA040423433360CB79DB0649D52A4A5F
:1008D000AF08136843F0010313601368244A03F060
:1008E0000103A2F57E742B4A0193019B54F827B0B3
:1008F000904205D0284A009B904208BF012300E0A7
:1009000000230AF00C060F2202FA06FCB3402BEA81
:100910000C024FF00F0C1A4344F82720144C4F6878
:10092000FA03226854BF22EA0E0342EA0E03236050
:10093000BA03626854BF22EA0E0342EA0E03636000
:10094000FA02A26854BF22EA0E0342EA0E03A36031
:10095000084BBA021A6854BF22EA0E0242EA0E029B
:100960001A600AF1040A013555E700BF0010014082
:10097000000401400C040140181002400000111056
:1009800000001210000021100000221000003110A1
:100990000000321000080140000C0140806808404F
:1009A00018BF01207047C26814230A4208BF1023F1
:1009B000C1507047002A08BF090401617047000058
:1009C00005480068704700BF1A48034900780A6864
:1009D00010440860704700BFF009002080B58048CF
:1009E000016841F010010160032000F051F80F2070
:1009F00000F004F800F022F8002080BD70B50D4E24
:100A000004464FF47A713078B1FBF0F081490968FF
:100A1000B1FBF0F000F0AAFA01250F2C08D838B984
:100A20004FF0FF3021460022002500F015F87460D9
:100A3000284670BD040000200C0000207047000014
:100A4000002806D4734600F09DFB9E46014A42F8FA
:100A50002010704700E100E070B5134B4FF0FF35F8
:100A60001B68C3F30223DC1E83F0070338BF002496
:100A700005FA04F6B243042B28BF042305FA03F356
:100A80009943A1401143BDE8704001F00DBB00BF88
:100A900005494FF6FF030A681A4060F30A2203482B
:100AA00010430860704700BF0CED00E00000FA053D
:100AB0002DE9F84300286CD0884649490446086867
:100AC00000F0070040450AD2086820F0070040EA1D
:100AD00008000860086800F00700404559D1206808
:100AE0005B4B8946810711D5410703D5196841F44D
:100AF000E0611960010703D5196841F4605119607C
:100B0000A1681A6822F0F00211431960C00737D1BA
:100B1000D9F8000000F0070040450DD9D9F80000D1
:100B200020F0070040EA0800C9F80000D9F80000EA
:100B300000F0070040452CD12068410705D5E16849
:100B40001A6822F4E06211431960000706D5206993
:100B5000196821F4605141EAC00018601C4600F099
:100B60005DF821681F4AC1F30311515CC84029494F
:100B700008601D480068FFF741FF0020BDE8F883CA
:100B80006068022808D0012825D153F8041C890385
:100B900006D40120BDE8F88353F8041C8901F8D578
:100BA00019681D4621F0030108431860FFF708FF8C
:100BB000064641F28837606829682B4601F00C012F
:100BC000B1EB800FA4D0FFF7FBFE801BB842F2D937
:100BD0000320BDE8F88353F8041C8907D9D5DFE763
:100BE000002002403C2C000808000020DD48184985
:100BF000094A00680968C1F30221515CC840704786
:100C0000D8481349044A00680968C1F3C221515CFD
:100C1000C84070470C0000204C2C000810B50C494F
:100C20000C480A6802F00C03082B07D1C2F3834377
:100C300009A4D203E35C02D40C48584310BD0968F0
:100C400009A25843C1F34041515CB0FBF1F010BD23
:100C50000410024000127A00020304050607080986
:100C60000A0B0C0D0E0F10100102000000093D00D0
:100C70002DE9FC41002800F09C8004460078B74E26
:100C8000C0071FD0706800F00C00042814D000F0DA
:100C900094FA02D17068C0030ED46068002800F096
:100CA0001481B0F5A02F00F02181B0F5803F00F055
:100CB000218100F045FA20E13068800302D56068A8
:100CC000002876D02078800716D5706810F00C0FB9
:100CD00005D000F072FA24D17068C00321D43068C6
:100CE000800702D52069012863D16069316821F04D
:100CF000F80141EAC00030602078000741D5A069C2
:100D000010B397480121C0F88014FFF759FE05463B
:100D1000706A800728D4FFF753FE401B0228F7D9DA
:100D2000F8E021698E48002900F08E8001210160E1
:100D3000FFF746FE054630688007D6D4FFF740FE31
:100D4000401B0228F7D9E5E085480021C0F880144F
:100D5000FFF736FE0546706A800712D5FFF730FEB2
:100D6000401B0228F7D9D5E07E484FF4FA510068BD
:100D7000B0FBF1F0019000BF0198411E00280191E5
:100D8000F9D12078400717D4E7697FB100F015FA50
:100D90003CD1012F0DD0216A706800F480328A4264
:100DA00007D1616A00F47010884202D10020BDE8CA
:100DB000FC810120BDE8FC81F06910F0805808D169
:100DC000F06940F08050F061F06900F080500090D0
:100DD0000098654F3868C0050FD4386840F48070BB
:100DE0003860FFF7EDFD05463868C00505D4FFF70C
:100DF000E7FD401B6428F7D98CE0E068A0B3052824
:100E000044D0012846D000F0C4F946E054490020FF
:100E100088460866FFF7D4FD0546022F0AD14746EB
:100E20003068800179D5FFF7CBFD411B03200229F3
:100E3000F6D9BCE730688001B8D5FFF7C1FD411B8A
:100E400003200229F6D9B2E700210160FFF7B8FDBF
:100E50000546306880077FF54FAFFFF7B1FD411BB6
:100E600003200229F5D9A2E700F093F93062FFF7D9
:100E7000A7FD054641F28837306A80071CD5FFF789
:100E80009FFD411B0320B942F6D990E7306A40F03C
:100E900004003062306A40F001003062FFF790FDDC
:100EA000054641F28837306A800705D4FFF788FD90
:100EB000401BB842F7D92DE0B8F1000F7FF464AFC2
:100EC000F06920F08050F0615EE700F039F93060A1
:100ED000FFF776FD0546306880037FF5F3AEFFF738
:100EE0006FFD411B03206429F5D960E7306840F4A9
:100EF00080203060306840F480303060FFF760FD63
:100F00000546306880033FF5DDAEFFF759FD401B15
:100F10006428F6D90320BDE8FC81206AB0F5803F43
:100F200005D1A168726822F4003211437160616AD0
:100F30000843716821F47411084370600120386619
:100F4000FFF73EFD0446306880013FF52FAFFFF705
:100F500037FD011B03200229F5D928E700100240C4
:100F6000000042420C00002000700040411E0020A2
:100F7000B0EB116F1CBF01207047044AF023516091
:100F800003490B70072190601160704710E000E08A
:100F900023ED00E090B110B5044690F8390008B98F
:100FA00000F0FFF800F0D4F82068016921F49041C6
:100FB0000161416921F02A0100F004B90120704764
:100FC0007047FEE710B586B04648114C016841F005
:100FD00010010160006800F01000019003200590EE
:100FE0000120CDE903004FF400500290019802A9BE
:100FF0002046FFF7FFFB20464FF400510122FFF788
:10100000D9FC0020322100F071FC06B010BD00BFF9
:101010000010014010B50E4C207808B1012010BD21
:101020004548FF214FF47A7200F0DCF810B101203E
:10103000207010BD207810BD80B501460448002204
:1010400002703D484FF47A7200F00EF9C0B280BDD4
:10105000E8090020F0B58BB02049214D4022052041
:10106000102320244FF48066C1E90A45C1E90C35FC
:10107000C1E90E20304C05F580630846C1E90865DA
:101080008026C1E9042540F81C3FC1E900652160C4
:10109000886100F047FB13480127016841F0040113
:1010A0000160006800F0040006900320CDE90767A6
:1010B0000A90069807A92846FFF79CFB0021072203
:1010C000FF200023CDE90077CDE90221064ACDE9D2
:1010D0000410204600F08EFA0BB0F0BD4400002052
:1010E00000080140181002408050DE19B0B50546D6
:1010F000FFF790FF50B1104800F0EEF830B1044611
:101100000D482946224600F095FA00E000242046CA
:10111000B0BD00BFB0B5054608460C46FFF78CFFD2
:1011200040B10548294622464FF47A7300F000F991
:101130000120B0BD0020B0BD88000020FEE7704750
:10114000306820F480303060306820F480207047B0
:10115000242084F839002068C16821F40051C1605E
:10116000204600F087BD01900320059002A80EC024
:1011700001987047064600680F4600211C46154638
:1011800000F022BA00F01F010122400902FA01F129
:101190007047306A20F001003062306A20F00400AD
:1011A0007047002084F838002046FFF709BF154635
:1011B0000E460446417500F02BB9706800F00C0033
:1011C000082870474161C16841F40051C1600020A6
:1011D0002021E06384F8391084F83A1010BD70477C
:1011E00070470000F8B5FFF7E2FFD44F20464D21CD
:1011F0008422B84720462421FF22B84720464021B8
:101200000122B847204611213F22B847204600F06E
:10121000FBF8204622213246B84720460F2100F035
:10122000CDF8024620460D21B847204601218D22E7
:10123000B847002084F8170120461821013D00F02E
:10124000BDF8400704D43DB1012000F08BF9F3E76D
:101250000320A0750120F8BD206800F085F9204624
:1012600000F0D6F80020F8BDF8B5FFF7A0FFB34FA7
:1012700020464D218722B847204624210022B84726
:10128000204640214122B847204600F0BDF82046C4
:101290001121F722B847204622213246B84720467E
:1012A0000E2100F08BF8024620460D21B84720465B
:1012B000222100F083F8B04209D0013DF7D1206827
:1012C00000F052F9204600F0A3F80020F8BD0220FB
:1012D000A0750120F8BD00BF70B50446407C28B160
:1012E0002046132100F06AF8054600E0657DEDB167
:1012F00004F117064FF480713046FEF76DFF20466B
:10130000102100F05BF8024620460D2100F065F840
:101310002046002132462B4600F022F8204684F871
:10132000175100F071F894F8170170BD002070BDDE
:1013300010B513460A460021044600F027F820465F
:1013400001218B2200F049F82046122100F036F8E6
:10135000204600F059F8204600F085F9012010BD24
:101360009BB1F8B5FFF706FF3068394600F014F975
:1013700030682CB100F01CF905F8010B013CF7E7CF
:101380000121BDE8F84000F01FB97047022B38BFBB
:101390007047F8B5FFF7EEFE306847F0800100F0C7
:1013A000FBF830682CB115F8011B00F0F5F8013C92
:1013B000F7E70121BDE8F84000F006B9B0B50446F2
:1013C000006800F0E9F8206800F0F2F805462068AF
:1013D000012100F0F9F82846B0BD70B50646006856
:1013E0000D460021144600F0EFF8306845F080010A
:1013F00000F0D2F83068214600F0CEF830680121C4
:10140000BDE8704000F0E0B81221FF22FFF7E5BF11
:101410007CB5044600F01EF90F2000F0A3F820462A
:1014200000F09CF8D4E90201434A0023C90441EAD0
:101430005031C004FEF776FE010A8DF80700000C5B
:101440000DF1050203238DF806108DF805002046E6
:101450000621FFF79BFF394D204639213422A8474A
:10146000207C37A10A5C20460921A84720460B2191
:101470000B22A84720460C212322A847A07C31A399
:10148000E27C617C185C32A39A5C520002EB001093
:1014900099B1C2B220461D21FFF79FFF607C2D4A03
:1014A000217D105C2C4A515C890001EB00101E214B
:1014B000C2B22046FFF791FF21E040F001001D215C
:1014C000C2B22046A847607C224A217D105C224A95
:1014D000515C890001EB00101E210330C2B220468E
:1014E000A84720463121FFF769FF00F0F8003121BD
:1014F000421D2046A847204637210C22A8472046F7
:1015000026210422A84720461F210822A84720465A
:10151000202100220026A847204621210822A84792
:10152000204641210122A84784F817612046BDE8E2
:101530007C4000F098B800BF0048E801DB130008C9
:10154000FFFCF9F600010203040506070809000084
:1015500001020304542C00086F2C0008012188228A
:10156000FFF73BBFFFF7D6B810B504463048006818
:1015700000F0FBF8218860680022FFF71BFA0120C9
:10158000FFF7C8F8218860680122FFF713FA64208A
:10159000BDE81040FFF7BEB8B0B5254D0C46286831
:1015A00000F06AF828682146BDE8B04000F0E2B8D3
:1015B00010B51F4C206800F05FF820680021BDE8DE
:1015C000104000F0D7B800BF19480129006818BFC3
:1015D00000F052B800F0C9B810B5044614480068CD
:1015E00000F0C3F8218860680122BDE81040FFF7D1
:1015F000E1B900BF70B5064600680D491C461546A6
:10160000806908603068FFF7E7FFC6E9025409986F
:101610007075089830750798F0740698B07405983E
:101620007074049830743046BDE87040FFF7F0BE27
:10163000EC090020B0B590F817510A46044600F1B5
:10164000170110462A46FEF7AEFD002084F8170168
:101650002846B0BD10B5012108220446FFF7BDFEA3
:101660000020A07510BDB0B5012109220446012556
:10167000FFF7B3FEA575B0BD818B80690022FFF72F
:1016800099B9000010B586B0234C20444FEAB02031
:1016900003280FD8DFE800F002101E2C1F48046852
:1016A00044F004040460006800F00400FFF75BFDF0
:1016B0001B482AE000202CE01848046844F0080485
:1016C0000460006800F00800FFF74DFD144800F5C5
:1016D00080601AE01148046844F010040460006857
:1016E00000F01000FFF73FFD0D4800F500600CE032
:1016F0000A48046844F020040460006800F02000F8
:10170000FFF731FD064800F5406002A9FFF772F8C7
:10171000012006B010BD00BF00F8FEBF1810024047
:101720000008014010B504460068012200236168EA
:10173000FFF7A8FFB8B1D4E9020101220023FFF7A7
:10174000A1FF80B1D4E9040100220123FFF79AFF31
:1017500048B1D4E9060101220023FFF793FFB0FA54
:1017600080F0400910BD012010BD818B80690122ED
:10177000FFF720B92DE9F047DFF86080DFF860A0BF
:101780000C4605464FF000090027072F22D8A988EC
:1017900028680022C047286AD047E2B2A989A86811
:1017A000D209C047286AD047A98828680122C047C3
:1017B000286AD047A98A2869FFF7F0F80646286A00
:1017C000D047701E01376400B0FA80F0400940EA4B
:1017D0004909DAE75FFA89F0BDE8F087B509000842
:1017E0003D070008012181F31088002247498968DC
:1017F00082F31088081A6FF00041B8BF08447047A0
:10180000012080F3108800214048806881F310880F
:10181000704700BF80B5FFF7D7F83C48007818B193
:10182000BDE8804000F002B880BD00BF10B5374869
:10183000C16829B1C1680139C16004BF012181704B
:101840000021012224290ED043185C694CB15C6947
:10185000013C5C6105D15A741C7C012C04BF9C695D
:101860005C610C31EEE78168013181608168013192
:1018700004BF0021816041780131CAB2092A88BFC2
:1018800000214170818801318AB2D2087C2A88BF48
:101890000021818010BD00BF10B51C48002100222E
:1018A000242A06D083180C3259619961597419742D
:1018B000F6E70B494FF47A720968B1FBF2F14A1E60
:1018C0000021B1EB126F07D1064BF0245A60064A93
:1018D00014709960072119600121017010BD00BFCB
:1018E0000C00002010E000E023ED00E0012282F374
:1018F000108800EB4000054A02EB800041618161E5
:1019000000214174017481F3108870471000002099
:10191000B0B590B00BA81421FEF75EFC4FF4E010B8
:10192000002402250A904FF48030CDE90644CDE929
:10193000044408950990CDE902040120019001A812
:10194000FFF796F970B90F200F940D940C950221B2
:101950000B904FF480600E900BA8FFF7A9F828B900
:1019600010B0B0BD03482721FEF72AFF01483321FC
:10197000FEF726FF712C00080E480F4A016841F05F
:1019800001010160416811400C4A41600168114049
:101990000160016821F480210160416821F4FE01A9
:1019A00041604FF41F01816005484FF00061016004
:1019B000704700BF001002400000FFF8FFFFF6FE76
:1019C00008ED00E080B582B08DF807009DF80700B3
:1019D000FEF780FE0090009808B9FFE707E0009945
:1019E0000020C8820099088300994883FFE702B06D
:1019F00080BD000080B582B08DF807009DF807001B
:101A0000FEF768FE0090009808B9FFE707E000992C
:101A1000002008820099488200998882FFE702B07E
:101A200080BD000080B584B08DF80E0002919DF855
:101A30000E00FEF74FFE0190019820B9FFE700204D
:101A40008DF80F0006E00198029900F06BF98DF80F
:101A50000F00FFE79DF80F0004B080BD80B596B081
:101A6000FFE741F21800C4F20200016841F00401EE
:101A70000160006800F0040011901198FFE7FFE793
:101A800041F21800C4F20200016841F00401016053
:101A9000006800F0040010901098FFE7FFE741F2A3
:101AA0001800C4F20200016841F48041016000683E
:101AB00000F480400F900F98FFE74FF400701290F1
:101AC000022013900120089014900320159040F6F6
:101AD0000000C4F20100069012A90791FEF78AFEE9
:101AE000069807994FF480621292FEF783FE089AD7
:101AF0002520099000210A91FEF7AEFF0998FEF714
:101B00009FFF0A9A43F60000C4F201000B904FF4C5
:101B1000E1310C2300F0EEF80B99086820F040004A
:101B20000860086820F02000086043F60C01C4F249
:101B30000101086840F020000860FFE741F218004A
:101B4000C4F20200016841F004010160006800F085
:101B500004000E900E98FFE7FFE741F21800C4F270
:101B60000200016841F004010160006800F0040017
:101B70000D900D98FFE7FFE741F21C00C4F2020050
:101B8000016841F400310160006800F400300C90FD
:101B90000C98FFE70420129002200290139001207D
:101BA00014900320159040F60000C4F2010000904C
:101BB00012A90191FEF71EFE0098019908221292C7
:101BC000FEF718FE029A2620039000210491FEF7EA
:101BD00043FF0398FEF734FF049A44F20040C4F236
:101BE000000005904FF4E1310C2300F083F80599D3
:101BF000086820F040000860086820F020000860B5
:101C000044F20C41C4F20001086840F02000086072
:101C100016B080BD80B500F0F5F9FFF71FFF80BD5D
:101C200080B584B08DF80F000291ADF806209DF8C4
:101C30000F00FEF74FFD0090009808B9FFE706E09F
:101C400000980299BDF8062000F06AF9FFE704B099
:101C500080BD000080B582B08DF807008DF80610B9
:101C60009DF807000DF106010122FFF7D9FF02B030
:101C700080BD0000B0B50446006804F108030ECB37
:101C8000056925F4405519432A4341F20C65026168
:101C9000C2686369AA4319431143C1604169A269DB
:101CA00021F44071114341611149884202D0FEF78D
:101CB0009DFF01E0FEF7A4FF19214843D4E900127B
:101CC0006FF063049200B0FBF2F06422B0FBF2F319
:101CD00003FB0400322404EB0010B0FBF2F000F030
:101CE000F00200F00F0002EB031210448860B0BD58
:101CF0000038014080B594B0139012911192109366
:101D0000139800901298019000200290039011996E
:101D1000049106901099059107906846FFF73AF9EB
:101D200014B080BD88B00290019101200490049805
:101D300080F310880298408BADF8020000200590D7
:101D4000059880F31088BDF8020020B9FFE7002055
:101D50008DF80F0025E002998868098B405C019995
:101D6000087001200690069880F310880299088B6D
:101D70000130088380B20299C989884204DBFFE7F9
:101D8000029900200883FFE70299488B01384883B5
:101D900000200790079880F3108801208DF80F002D
:101DA000FFE79DF80F0008B07047000080B586B0CF
:101DB0000590059800680068049005980068C06860
:101DC000039005980068406902909DF81000800615
:101DD000002830D5FFE70598006840688DF80700B7
:101DE0009DF80700059A9168D28A88540599C88A97
:101DF0000130C88280B20599C989884204DBFFE7B7
:101E000005990020C882FFE70598408B0599C9898C
:101E1000884205DAFFE70599488B01304883FFE7E0
:101E20000598C06930B1FFE70598C1699DF80700C2
:101E30008847FFE7FFE79DF810000006002836D529
:101E4000FFE79DF80C000006002830D5FFE7059855
:101E5000808A68B9FFE705980168C86820F08000AB
:101E6000C86005980168C86840F04000C8601DE07F
:101E70000599012081F8200005994868498A405C4D
:101E80000599096848600599488A0130488280B2FE
:101E900005998989884204DBFFE70599002048827B
:101EA000FFE70599888A01388882FFE7FFE79DF8F8
:101EB00010004006002830D5FFE79DF80C004006D2
:101EC00000282AD5FFE70598808A58B9FFE70598CA
:101ED0000168C86820F04000C8600599002081F8BA
:101EE000200019E005994868498A405C059909680D
:101EF00048600599488A0130488280B205998989ED
:101F0000884204DBFFE7059900204882FFE7059936
:101F1000888A01388882FFE7FFE706B080BD0000AD
:101F200088B003900291ADF806200020ADF80400BF
:101F3000FFE7BDF80400BDF8061088425ADAFFE753
:101F4000FFE701200490049880F310880398808AAA
:101F5000ADF8020000200590059880F31088BDF8C8
:101F6000020003998989884201DAFFE717E0BDF88A
:101F700002000399898988420FD1FFE7039800681E
:101F8000C0680006002807D4FFE703980168C86806
:101F900040F08000C860FFE7FFE7FFE7D1E7029865
:101FA000BDF80410405C039A5168128A88540120DD
:101FB0000690069880F310880399088A01300882F9
:101FC00080B203998989884204DBFFE703990020E6
:101FD0000882FFE70399888A0130888200200790F1
:101FE000079880F31088FFE7BDF804000130ADF8D2
:101FF00004009EE703980168C86840F08000C8604C
:1020000008B0704740F6A011C2F2000143F600008C
:10201000C4F20100086040F2A050C2F20000486023
:1020200040F2A010C2F2000088604FF400728A8172
:10203000CA81002008824882C88208834883888237
:10204000C86181F8200040F6C411C2F2000144F2D8
:102050000043C4F200030B6040F2A073C2F200031D
:102060004B6040F2A033C2F200038B608A81CA81C8
:1020700008824882C882088348838882C86181F8C0
:102080002000704780B540F6A010C2F20000FFF7B4
:102090008DFE80BD80B540F6C410C2F20000FFF78F
:1020A00085FE80BDFEE7000010B5074C00F00F0371
:1020B000B0F1FF3F034A2344C8BF831808011870DA
:1020C00010BD00BF00E400E014ED00E080B582B078
:1020D0000190009140F6E910C2F2000000789DF8EE
:1020E0000410FFF7B7FD019802B080BD9CB0FEF769
:1020F00075FC18B16A482A21FEF762FBFFF708FC5D
:10210000FEF738FBFFF7C8FBFFF784FDFEF75AFF29
:10211000FEF7A0FFFEF74AFB40204FF0010B4FF007
:10212000000832260FF2B4198DF86E0043F2232016
:10213000ADF86C0016AD1BA80321FEF7EBFF18B934
:1021400057484821FEF73CFB6420FEF7E3FAFFF70F
:1021500057FB8246FEF724FBFEF725FB5046FFF7B0
:1021600041FBB0F57A7F80F29280BBF1000F1DD168
:102170005FFA88F0C82100FB01F45046FFF732FBFC
:10218000A04213DBF9B20DF12600FEF714FB0DF1AE
:10219000250008F10108FEF70AFB38B19DF825007B
:1021A00040F004004F2808BF4FF0FF082846FEF714
:1021B0009DFF0028D2D00146142808D19DF8582050
:1021C000F0B2824203D19DF86800402803D048460F
:1021D00000F090F8C2E733484FF40051FEF7E3FBFC
:1021E00031A000F019FD1898FEF701F8044619987F
:1021F0000891FDF7FCFF824617980791FDF7F7FF5E
:10220000024608980B469DF858100094CDE9010A43
:102210000798039027A000F06DF8BBF1000F17D1CD
:102220005FFA88F0FF2813D0F9B20DF12600FEF70F
:10223000C2FA0DF12500FEF7BAFA28B19DF8250083
:1022400040F004004F2803D0C820FEF763FAEBE704
:102250001798FDF7CCFF824618988846FDF7C7FF10
:10226000834619980F46FDF7C2FF9DF85820CDE927
:1022700004010DF1260014A1CDE900A8CDE902B7B3
:1022800000F048F8471C4FF000084FF0000B0136F3
:10229000F0B2352888BF32268DF86D604BE700BF5D
:1022A0005B2C000800100140476574206461746174
:1022B0003A000000256326252E316626252E31663C
:1022C00026252E3166260A00256326252E31662610
:1022D000252E316626252E316626000057726F6E38
:1022E0006720446174612C2053697A653A20256423
:1022F0000A0000000FB4054B10B503A9044A029868
:1023000000F0EEF810BC5DF814FB0000CD200008D2
:10231000000000200FB4084B10B504A902AA0398CE
:1023200000F0DEF8044602A9002000F070FC204610
:1023300010BC5DF814FB00000F2C000802E008C878
:10234000121F08C1002AFAD170477047002001E02F
:1023500001C1121F002AFBD1704700002DE9FF5F69
:1023600082B00021DDE90430020DDDF840B0034306
:1023700018D044F61050A2F2FF32424315141198BF
:1023800001281FD0A5EB0B00401C5FEA000A4FF0AC
:1023900000064E4FDFF83891B046504615D5CAF1C9
:1023A000000413E0119801244AA3012801D16FEA27
:1023B0000B010298119AC0E90031C0E9024206B04F
:1023C000BDE8F09FCBF10000DFE704460021404A62
:1023D000491842EB0450CDE9001012E0E00707D0A5
:1023E00032463B4640464946FDF7E0FF8046894677
:1023F00032463B4610461946FDF7D8FF06460F46C3
:102400006410002CEAD1DDE90401DDE90023BAF112
:10241000000F06DAFDF7CAFF42464B46FDF7C6FF3E
:1024200005E0FEF735F842464B46FEF731F8044624
:102430000E460022284BFEF7B3F803D84FF0FF30CA
:10244000014607E00022254B20463146FDF707FFF5
:10245000FEF78DF8102409E0002C0ADB0A22002385
:10246000FDF760FE039B30321A55641E50EA0102EC
:10247000F2D1641C039AC4F111031444119A012A85
:1024800003D0012208430DD10AE0084304D0002004
:102490004FF0110B119072E7A3EB0B056D1E0DE0D1
:1024A0005B4504DD4FF0000205F1010504E003DAAD
:1024B0004FF00002A5F10105002AECD00298119915
:1024C000C0E90231C0E9004579E70000000014408E
:1024D0000000F03F300000000000F0430000E03F4B
:1024E0002DE9FF4F95B09B468946064600250FE231
:1024F000252877D100242746F84A0121059400E0D9
:10250000044316F8013F203B01FA03F01042F7D1D3
:1025100030782A2811D06FF02F033078A0F13002E4
:10252000092A16D8059A44F0020402EB820203EB52
:1025300042021044761C0590EFE759F8042B0592EF
:10254000002A03DA504244F40054059044F0020497
:10255000761C30782E2816D116F8010F44F00404AA
:102560002A280DD06FF02F023078A0F13003092B0C
:1025700009D807EB870302EB4303C718761CF3E780
:1025800059F8047B761C30786C280FD006DC4C2878
:1025900017D068280DD06A2814D104E0742810D010
:1025A0007A280FD10DE044F400140AE044F48014BA
:1025B00001E044F440147278824202D104F58014A0
:1025C000761C761C307866280BD013DC582877D020
:1025D00009DC002875D04528F6D04628F4D04728D5
:1025E0001AD19DE118E0632835D0642879D0652898
:1025F00012D195E1702873D008DC6728F1D06928E2
:102600006FD06E280DD06F2806D1B5E073282CD07E
:10261000752875D0782874D05A46179990476D1C44
:1026200075E1C4F30250022809D003280DD0D9F86F
:10263000001004280DD00D6009F1040967E1D9F8F4
:102640000010EA17C1E90052F6E7D9F800100D8032
:10265000F2E70D70F0E719F8041B8DF80010002068
:102660008DF80100EA46012003E059F804AB4FF071
:10267000FF3061074FF0000102D40DE008F10101C5
:102680008846B9420FDA8045F8DB1AF808100029AD
:10269000F4D108E008F1010188468142FADB1AF81A
:1026A00008100029F6D105985B46A0EB08072146E3
:1026B0003846179A00F094FA284400EB080507E022
:1026C0004DE029E10DE01AF8010B5A4617999047A1
:1026D000B8F10108F7D25B4621463846179A13E154
:1026E00042E00A220092C4F302524FF0000A022A8A
:1026F00008D059F804CB032A4FEAEC710AD00DE058
:1027000029E02AE009F1070121F00702F2E802C1FD
:10271000914609E00FFA8CFC4FEAEC71042A03D1D0
:102720004FFA8CFC4FEAEC71002907DA0A460021C7
:10273000DCF1000C61EB02012D2202E0220504D540
:102740002B228DF80420012203E0E20701D0202291
:10275000F7E7904659E00A2102E010220DE010212F
:102760004FF0000A00910BE010224FF0000A44F0F5
:1027700004040827009203E008224FF0000A0092A8
:10278000C4F30252022A05D059F804CB0021032ACF
:1027900008D009E009F1070121F00702F2E802C1BF
:1027A000914605E01FFA8CFC042A01D10CF0FF0CC5
:1027B0004FF00008220728D5702806D0009B83F030
:1027C000100353EA0A0305D00EE040228DF80420DE
:1027D000012208E05CEA010206D030228DF80420D4
:1027E0008DF8050002229046009B83F0080353EA0F
:1027F0000A030AD15CEA010201D1620705D5302241
:102800008DF804204FF001087F1E582804D034A012
:1028100003900EA802900DE036A0F9E753466046FB
:10282000009AFDF77FFC84460398825C0298401E64
:10283000029002705CEA0100F0D1029806A9081A21
:1028400000F1200A600702D524F4803400E001275B
:10285000574502DDA7EB0A0000E0002000EB0A016B
:10286000009005984144401A0590E00306D45B4669
:102870002146179A059800F0B3F90544002706E0B1
:1028800001A85A46C05D179990476D1C7F1C4745AB
:10289000F6DBE0030CD55B462146179A059800F05D
:1028A0009FF9054404E030205A46179990476D1C63
:1028B0000099481E00900029F5DC08E00298029972
:1028C0005A460078491C0291179990476D1CBAF13D
:1028D0000001AAF1010AF1DC65E10000092801000C
:1028E0003031323334353637383961626364656686
:1028F0000000000030313233343536373839414248
:10290000434445460000000000F058F90544761C99
:10291000307800287FF4ECAD19B02846BDE8F08F80
:10292000620700D4062709F1070222F0070CFCE831
:102930000223E14603F000485FEA080C02D00FF2E0
:10294000702C0DE05FEA045C02D50FF2682C07E002
:102950005FEAC47C02D00FF2602C01E0AFF2700C91
:102960004FF0FF3823F00043CDF850C065280CD05D
:1029700006DC452809D046281DD047283DD13DE03A
:10298000662818D067287ED138E00021112F01DB9E
:10299000112000E0781CCDE9000106A90EA8FFF780
:1029A000DDFCDDE90F010E9A03910021009207F191
:1029B000010A04914DE04FF000400097CDE901106D
:1029C00006A90EA8FFF7CAFCDDE90F0203920E9BD1
:1029D00011990022DDF80CA00093049211B9791C22
:1029E00000EB010AB7EB0A0004D4C0F1FF3007F195
:1029F000010A0490AAEB0700019044E0012F00DADD
:102A000001270021112F01DD112000E03846CDE91A
:102A1000000106A90EA8FFF7A1FCDDE90F010E9A3F
:102A20000391002104910092BA4621070CD4039926
:102A3000514500DA8A46BAF1010F05DD009AAAF184
:102A40000101515C302908D0B84202DA10F1040FBC
:102A500006DA0121CDE9011015E0AAF10101E9E74B
:102A6000002805DC049901440491AAEB000102E06E
:102A7000411C514500DD8A460499401A401C0190D2
:102A80004FF000400290200704D40198504501DB2C
:102A9000CDF8048000208DF84F0002980DF14F070B
:102AA000B0F1004F25D02B200E9002984FF0020875
:102AB00000280CDA404202902D200E9007E00A21F7
:102AC0000298FDF7A7FB3031029007F8011DB8F11D
:102AD0000001A8F10108F2DC02980028EFD1791E6C
:102AE0000E980870307800F0200040F0450007F89C
:102AF000020D12A8C01B00F107081498007800B15D
:102B0000012000EB0A01019801EBE07105984144B6
:102B1000401A401E0590E00306D45B462146179AF2
:102B2000059800F05DF805441498007818B15A46ED
:102B3000179990476D1CE00324D55B462146179AF0
:102B4000059800F04DF805441CE00498002807DBC8
:102B5000DDE90301884203DD0098405C179901E03C
:102B6000179930205A469047049805F10105401CFA
:102B700004900198401E019004D12E205A461799C6
:102B800090476D1CBAF10001AAF1010ADDDC05E0F5
:102B900017F8010B5A46179990476D1CB8F10001C0
:102BA000A8F10108F4DC5B462146179A0598ABE6CC
:102BB0002D0000002B000000200000002DE9F04156
:102BC000044600251E461746880404D405E039460D
:102BD0002020B0476D1C641EF9D52846BDE8F08161
:102BE0002DE9F041044600251E469046C80301D554
:102BF000302700E02027880404D505E04146384608
:102C0000B0476D1C641EF9D52846BDE8F0810A68FE
:102C1000531C0B601070704710B5044601E0FFF7BD
:102C200055FA14F8010B04490028F8D1BDE810400A
:102C30000A20FFF74BBA000000000020000000004F
:102C4000000000000102030406070809000000005C
:102C500001020304060708090A0B0C2E2E2F5573D8
:102C600065722F4D61696E2F6D61696E2E63000173
:102C7000002E2E2F53797374656D2F7379732F7314
:102C800079732E6300000000A82C000800000020CB
:102C9000100000003C230008B82C000810000020A1
:102CA000E81F00004C2300080000000001000000A5
:082CB000100000000024F400F4
:04000005080000ED02
:00000001FF
